:020000020000FC
:1000000014C079C075C0189518951895189518954D
:100010001895526F7373205768656E6D6F757468AD
:100020002031382F392F3230303400E808B900E061
:100030000EBBE09A0DB301BF01E00EBBE09A0DB21A
:1000400006B300FD6BC004E008BB03E007BB03E29E
:1000500007B900E305BFF89400E40BBF00E40ABF52
:1000600078948895B299F5CFC09AF89400E20BBFC6
:1000700000E20ABF7894889541D0B29BF6CFC39A2C
:10008000F8940DE806B908E205BF7894889505B1A3
:1000900037983398001570F0B39927C000E00FBD72
:1000A00005E80EBD08E900BF29D028D000E000BF58
:1000B000C1981BC000E00FBD04E60EBD08E900BFFB
:1000C0001DD01CD005E80EBD00E00FBD17D016D026
:1000D00004E60EBD13D012D005E80EBD00E00FBD42
:1000E0000DD00CD000E000BFC198C098C398B1CF2C
:1000F00000E00BBF189500E00BBF189514E612BF87
:1001000018B7126018BF15E013BF18B711FFFDCF65
:1001100018B7126018BF10E013BF08950CE008BBB9
:1001200002E007BB00E00FBD07E00EBD0FE00DBD14
:1001300005E600BFB39905C001B7039501BFDEDF37
:10014000DDDFB29905C001B70A9501BFD7DFD6DF61
:10015000B099F0CFF894E199FECF00E00EBB01B763
:100160000DBBE29AE19A00E000BF789403E207B980
:100170000DE806B908E205BFC1DFC0DFBFDF889523
:1001800005B0F894E199FECF01E00EBB0DBAE29AFA
:10019000E19A789401E007BBB1DFB0DFC09B02C0F9
:0801A000C098FACFC09AF8CF15
:00000001FF
